:100000000C945D000C94CA010C947A000C947A0054
:100010000C947A000C947A000C947A000C947A0078
:100020000C947A000C947A000C947A000C947A0068
:100030000C947A000C947A000C947A000C947A0058
:100040000C947A000C947A000C947A000C947A0048
:100050000C947A000C947A000C947A000C947A0038
:100060000C947A000C947A000902120001010080BD
:100070001909040000000000000012011001FF0037
:100080000008C016DC050401010200010E03550042
:10009000530042006100730070001C03770077007A
:1000A00077002E00660069007300630068006C0032
:1000B0002E00640065000403090411241FBECFEF65
:1000C000D8E0DEBFCDBF11E0A0E0B1E0E6E5F2E1AF
:1000D00002C005900D92A230B107D9F711E0A2E05D
:1000E000B1E001C01D92AC34B107E1F70E941709DD
:1000F0000C9429090C940000CF93DF9360912801A0
:10010000635067FD13C080912501CCE0D0E0C81B8F
:10011000D109C45DDE4F809124018D3209F458C0AD
:100120008091020187FD9DC01092280180910001FD
:1001300084FF41C0609101016F3F09F43CC0693008
:1001400008F470C06850609301018091180198E82C
:1001500089278093180168E08091020187FD1DC006
:10016000409126015091270186FF72C0FA01862F27
:10017000A9E1B1E094919D9331968150D9F7262F52
:10018000215030E02F5F3F4F240F351F3093270160
:1001900020932601C62FCC5F50C089E191E00E94D8
:1001A000D707682F893008F4A4C08FEF809301012E
:1001B000CEE1C093000194E183B1837031F491509A
:1001C000D9F71092290110922301DF91CF91089560
:1001D000683009F0A9CF83EC809318018AE58093F9
:1001E0000001109202018881807609F045C09A8151
:1001F00010922101898181114AC01092220121E2CD
:1002000031E082E030932701209326018F3FC1F136
:100210009F81911104C09E81981708F4892F8093C3
:10022000010182CF109201018091180198E889277D
:1002300080931801611190CFC4E089E191E00E94A0
:10024000C601CC3009F4B5CF8FEF80930101B1CF57
:10025000DA01862FE9E1F1E09D9191938150E1F778
:100260008ECFCE010E9447088F3FF9F0882309F412
:100270005BCF1092010158CFCE010E942306C6CF5A
:10028000988197FD16C090E890930201C8CF853001
:1002900091F0863001F18830D1F0893091F021E27F
:1002A00031E08A3021F180E0ADCF8EE18093000112
:1002B0003BCF8E81E8CF9093290121E231E080E0AD
:1002C000A1CF90932B0121E231E080E09BCF2BE284
:1002D00031E081E097CF8B81813001F18230B1F044
:1002E000833051F080E090E4909302018FCF81E061
:1002F00089CFC82FCC5FA1CF911118C086EB90E0B9
:10030000909327018093260184E0EDCF88E690E06A
:10031000909327018093260182E1E5CF8AE790E060
:10032000909327018093260182E1DDCF913051F037
:100330009230C1F68CE890E09093270180932601DB
:100340008EE0D1CF8AE990E0909327018093260137
:100350008CE1C9CFE9E6F0E0808183608083E89A90
:100360000895A82FB92F80E090E041E050EA609511
:1003700030E009C02D9182279795879510F084274A
:100380009527305EC8F36F5FA8F30895EADF8D9379
:100390009D930895CF93CFB7CF93C395189BE9F75B
:1003A000189B09C0189B07C0189B05C0189B03C069
:1003B000189B01C0A1C0DF93C0912501DD27C45D5A
:1003C000DE4F189B02C0DF91EBCF2F930F931F934B
:1003D00003B12FEF00FB20F94F933F9313B14FEF81
:1003E000012700FB21F93BE031C04E7F012F13B103
:1003F000216028C0102F4D7F2260000003B129C06A
:100400004B7F2460012F000013B12BC013B1477F35
:1004100028602AC04F7E03B120612CC04F7D13B1EC
:1004200020622FC04F7B03B1206432C0422703B14A
:1004300049934FEF0000102710FB20F913B1137000
:10044000C9F1297F91F2012700FB21F903B1237F34
:1004500089F2315058F1102710FB22F913B1277E91
:1004600079F2012700FB23F92F7C81F203B11027D9
:1004700010FB24F92F7971F200C013B1012700FBA2
:1004800025F92F7359F200C003B1102710FB26F98C
:10049000223040F200C013B1012700FB27F92430BD
:1004A00028F64F77206813B10000F9CF11E01CBB8C
:1004B000002717C03B503195C31BD04011E01CBB37
:1004C0000881033CE9F00B34D9F020912301198114
:1004D000110F1213EDCF093641F10D3211F0013E2B
:1004E00039F700932A013F914F911F910F912F915E
:1004F000DF91CCB3C0FD51CFCF91CFBFCF91189535
:1005000020912A01222379F310912801112311F55A
:10051000343012F1309328012093240110912501E9
:100520003BE0311B3093250117C0009128010130B9
:100530008CF40AE53091000134FD10C000930001F5
:10054000C8E1D1E00FC02795A8F45150A9F4220FBB
:100550000000F9CF4AE503C042ED01C0432FC4E1DA
:10056000D0E032E014B11360289A14B905B120E448
:1005700013E05F93012756E005B9279520F4515009
:1005800021F4220FF9CF012756E000003B5A05B9AC
:10059000D0F2279528F4515029F4220F0000F9CF0A
:1005A000012756E0279505B920F4515021F4220F78
:1005B000F9CF012756E02991332305B921F60C7FA5
:1005C00010912901110FC651D04005B911F01093B7
:1005D000230111E01CBB016014B11C7F402F4C7F34
:1005E0005F9100C000C005B914B945B97CCF682F30
:1005F00058E080E0709148012091470167FD1EC0DE
:100600002B98660F880F1C998F5F2D9A36B5472F50
:10061000415030F096B5931B9217E0F34150D0F75C
:100620002D9836B5472F415030F096B5931B921751
:10063000E0F34150D0F7515009F708952B9AE1CFDC
:100640008EBD0DB407FEFDCF8EB5089521E19695C0
:100650008795779567952A95D1F7209146012617BA
:10066000D9F060934601E0914301F09144018DE49B
:100670000995E0914301F091440180E00995E091F2
:100680004301F0914401809146010995E0914301B5
:10069000F091440180E009940895809145018CBD5A
:1006A000809142018DBD08958823C1F0883008F003
:1006B00042C027EF32E0309344012093430191E0A0
:1006C00090934801843039F1D8F0863049F158F1DF
:1006D0008730D1F483E080934701089580E293E06E
:1006E000909344018093430181E08093470180937C
:1006F000480182E58093450181E08093420108959D
:10070000823069F0833099F080E68093470182E07F
:1007100080934801089588E180934701089580E619
:100720008093470108958CE080934701089580E30A
:1007300080934701089520E233E0309344012093F1
:1007400043011092420191E0909347019093480138
:10075000893039F050F4883061F683E580934501A3
:10076000089582E58093450108958B3049F08C30DF
:1007700009F0BFCF81E58093450190934201089530
:1007800081E580934501089526B530914801909107
:100790004701315030F086B5821B8917E0F33150A4
:1007A000D0F7089584B18C6284B92A982D9826B523
:1007B00030914801432F90914701415030F086B568
:1007C000821B8917E0F34150D0F72A9A26B53150A1
:1007D00030F086B5821B8917E0F33150D0F72A98A4
:1007E00080914301909144018052934019F01092FE
:1007F00046010895809145018CBD809142018DBDD7
:1008000010924601089584B1837D84B985B1837DBA
:1008100085B91CBC0895CF93DF93C0E2E0914301FA
:10082000F09144018CEA0995E0914301F091440173
:1008300083E50995E0914301F091440180E0099539
:10084000D82FE0914301F091440180E00995D33520
:1008500009F43AC01CBC26B530914801432F909151
:100860004701415030F086B5821B8917E0F34150B3
:10087000D0F72A9A26B5432F415030F086B5821B17
:100880008917E0F34150D0F72A9826B5315030F05F
:1008900086B5821B8917E0F33150D0F7E091430110
:1008A000F091440183E0E032F80739F0C15009F0DB
:1008B000B9CF81E0DF91CF910895809145018CBD42
:1008C000809142018DBDF2CF80E0DF91CF910895FC
:1008D000CF92DF92EF92FF926B017C010E94260380
:1008E000D701C60181709927AA27BB27880F880FD7
:1008F000880FE0914301F091440180620995D7018E
:10090000C60139E0B695A795979587953A95D1F7A1
:10091000E0914301F09144010995D701C601B695D4
:10092000A79597958795E0914301F091440109952A
:10093000E0914301F091440180E0FF90EF90DF905F
:10094000CF900994CF92DF92EF92FF920F931F9373
:10095000CF93DF936B017C01C42FD22F0E9426031B
:10096000970186010170112722273327802F880FD6
:10097000880F880FE0914301F0914401806409954C
:10098000D701C60159E0B695A795979587955A95D1
:10099000D1F7E0914301F09144010995D701C601D7
:1009A000B695A79597958795E0914301F0914401FD
:1009B0000995E0914301F09144018C2F0995DD23C5
:1009C000B9F0CF3791F0D6B5CEE1C701B6010E949C
:1009D00068048F3769F486B58D1B8D3310F0D6B55A
:1009E000C150C111F2CF81E004C08FE00E94AE057A
:1009F00080E0DF91CF911F910F91FF90EF90DF90FA
:100A0000CF900895CF92DF92EF92FF920F931F93B2
:100A1000CF93DF931F92CDB7DEB76B017C01498383
:100A20000E942603E0914301F09144018CE4099572
:100A3000D701C60179E0B695A795979587957A95E0
:100A4000D1F7E0914301F09144010995D701C60126
:100A5000B695A79597958795E0914301F09144014C
:100A60000995E0914301F091440180E009954981A5
:100A70004F3FE9F006B51EE1C701B6010E946804C8
:100A80008F3F99F486B5801B8D3310F006B5115059
:100A90001111F2CF81E00F90DF91CF911F910F9153
:100AA000FF90EF90DF90CF90089580E0F4CF8FE03B
:100AB0000E94AE0580E0EFCF1F93CF93DF931F928C
:100AC000CDB7DEB7182FE0914301F091440180EAE1
:100AD00099830995E0914301F09144019981892F0F
:100AE0000995E0914301F0914401812F0995E0912E
:100AF0004301F091440180E00F90DF91CF911F916D
:100B000009941F93CF93DF9300D0CDB7DEB7182F92
:100B1000E0914301F091440180EC6A839983099547
:100B2000E0914301F09144019981892F0995E09169
:100B30004301F0914401812F0995E0914301F09127
:100B400044016A81862F09958EE10E94AE0580E0FE
:100B50000F900F90DF91CF911F910895882349F056
:100B600030E026B596B5921B9C33E0F33F5F381317
:100B7000F8CF0895259A23982B9A50E217D05A95CA
:100B8000E9F70895AC0188E605D0842F03D089E603
:100B900001D0852F0FD028E030E0382780FB8695E4
:100BA00006D02A95D1F730FB02D000D06894239864
:100BB0002B9A16F02B98239AE0914A01F0914B0161
:100BC0003197F0F72D9AE3B1E3FBE0914A01F09100
:100BD0004B013197F0F72D98089520ECE7DF46F4AC
:100BE0002A95E1F780E02AE1E5DF2A95E9F7DECFF3
:100BF00028E030E0DBDF869587F938272A95D1F7A2
:100C0000D5DF27F9322772F3D1DFD0CFDB01742F84
:100C1000B9DF84E2BFDFE1DF8D937A95D1F70895E4
:100C2000DB01742FAFDF83EFB5DF8DE1B3DF84E647
:100C3000B1DF8D91AFDF82E7ADDFCFDF8078D9F70D
:100C40007A9589F70895CF93DF93EC0189818130FC
:100C500089F1823009F4ABC0833009F461C084307B
:100C6000B1F1873009F482C0853009F402C18630C1
:100C700009F4A2C0883009F4D5C0893009F4FFC056
:100C80008A3009F42AC18B3009F456C18C3009F43A
:100C900069C18D3009F480C18E3009F483C18F3071
:100CA00009F4FEC0803109F41FC18F3709F439C13E
:100CB00080E02DC0329B56C0809103010E945403F6
:100CC0001092040141980E94D20380E020C08091DC
:100CD0000401811110C05B8140E08A81482B6627A6
:100CE00057FD6095762F40930D0150930E01609350
:100CF0000F01709310019F8180E02E81822B9093D1
:100D000012018093110182E0809313018FEF25E09F
:100D100031E03093270120932601DF91CF91089590
:100D2000E0914301F09144018A8109958093050186
:100D3000E0914301F09144018B8109958093060174
:100D4000E0914301F09144018C8109958093070162
:100D5000E0914301F09144018D8109958093080150
:100D600084E0D5CF85E00E945403AACF809104018E
:100D7000811110C05B8140E08A81482B662757FDB6
:100D80006095762F40930D0150930E0160930F01F3
:100D9000709310019F8180E02E81822B909312012D
:100DA0008093110183E0809313018FEFB0CF0E94F5
:100DB0000304419A80E0ABCF80910401811110C0FF
:100DC0009B8180E02A81822BAA2797FDA095BA2FCC
:100DD00080930D0190930E01A0930F01B093100129
:100DE0003C812D81822F8F7080931601822F807F0E
:100DF00040E1849FC0011124830F911D9093150140
:100E00008093140120FD809317019F8180E02E8143
:100E1000822B909312018093110181E08093130142
:100E20008FEF75CF80910401811110C09B8180E00C
:100E30002A81822BAA2797FDA095BA2F80930D01B6
:100E400090930E01A0930F01B09310011092150121
:100E500010921401109216019F8180E02E81822B46
:100E6000909312018093110184E0809313018FEF1E
:100E70004ECF0E940B048093050181E048CF81E0B2
:100E8000809304018A819B81AC81BD8180930D0197
:100E900090930E01A0930F01B093100180E037CF23
:100EA0009B8180E02A81822BAA2797FDA095BA2FEB
:100EB00080930D0190930E01A0930F01B093100148
:100EC0009F8180E02E81822B9093120180931101EB
:100ED00085E0809313018FEF1ACF8A8180930301FD
:100EE0001092050181E013CF9B8180E02A81822B43
:100EF000AA2797FDA095BA2F80930D0190930E011C
:100F0000A0930F01B09310019F8180E02E81822B6E
:100F1000909312018093110186E0809313018FEF6B
:100F2000F6CE81E080930501109206011092070130
:100F30001092080184E0EBCE9B8180E02A81822B15
:100F400090934B0180934A012A9A229A83E00E944F
:100F5000AE052A98419880E10E94AE050E94BA052C
:100F600080E0D5CE80EC0E94CA0580E00E94CA05D0
:100F70008AE00E94AE052A9A85E00E94AE052A9872
:100F800085E00E94AE0584B1837D84B985B1837DFF
:100F900085B9419A80E0BBCE0E94ED0580930501A2
:100FA00081E0B5CE8A810E94CA0580E0B0CE0F9361
:100FB0001F93CF93DF93582F792F062F2091130182
:100FC000322F3250323050F0253009F443C00FEF49
:100FD000802FDF91CF911F910F910895662391F19A
:100FE00080910D0190910E01A0910F01B09110011F
:100FF000C52FD72F10E01CC00E945C05888380910C
:101000000D0190910E01A0910F01B0911001019678
:10101000A11DB11D80930D0190930E01A0930F01AE
:10102000B09310011F5F2196101751F0209113010A
:10103000223011F7BC01CD010E9468048883DFCF04
:10104000083030F610921301802FDF91CF911F915D
:101050000F910895462F682F80910D0190910E01F8
:101060000E94060680910D0190910E01A0910F0142
:10107000B0911001800F911DA11DB11D80930D0134
:1010800090930E01A0930F01B0931001A1CFFF9296
:101090000F931F93CF93DF93382F792F162F209123
:1010A0001301213071F0243061F0263009F490C032
:1010B000FF24FA948F2DDF91CF911F910F91FF9014
:1010C0000895112309F4B1C080910D0190910E0192
:1010D000A0910F01B0911001C32FD72F00E0F12C88
:1010E00050C02091140130911501232B09F053C0F9
:1010F00021E04881BC01CD010E94A2042091110190
:1011000030911201215031093093120120931101C5
:10111000232BE9F4109213018091160181FF38C04E
:101120002091170130E0809114019091150128174A
:10113000390771F160910D0170910E0180910F01DD
:101140009091100148810E940205FF24F394809140
:101150000D0190910E01A0910F01B0911001019627
:10116000A11DB11D80930D0190930E01A0930F015D
:10117000B09310010F5F2196011709F49BCF2091C6
:101180001301213009F4ADCF68810E948105B6CFEB
:10119000FF24F394DCCF20E04881BC01CD010E9404
:1011A000A204809117018150809317018111A6CF6D
:1011B00060910D0170910E0180910F0190911001CD
:1011C00048810E940205809114018093170196CFF7
:1011D000462F682F80910D0190910E010E941006FC
:1011E00080910D0190910E01A0910F01B09110011D
:1011F000810F911DA11DB11D80930D0190930E01D2
:10120000A0930F01B09310018091110190911201F0
:10121000811B91099093120180931101892B29F46C
:1012200010921301FF24F39445CFF12C43CF1BB848
:1012300015B88BEF8AB98FEF84B914B883E087B9FA
:101240009EEF98B985BD0E94AA0178940E947C0007
:06125000FDCFF894FFCF72
:021256005AFF3D
:00000001FF
